:1000000097C0A6C0A5C0A4C0A3C0A2C0A1C0A0C0E4
:100010009FC09EC0B3C19CC09BC09AC099C07C1FAA
:1000200002200220022002207C1F000000000000AD
:10003000000000007C1F001F82208220822082207E
:100040007C00000082208220822082207C1F7C0095
:1000500080008000800080007C1F7C008220822045
:1000600082208220001F7C1F82208220822082200A
:10007000001F7C0002000200020002007C1F7C1FA7
:1000800082208220822082207C1F7C00822082208D
:10009000822082207C1F0000F03F8C0082008C00B8
:1000A000F03F0000FE07001800200018FE070000C7
:1000B000FE1F0020001F0020FE1F0000FE3F000169
:1000C00080008000003F0000803F8000803F800073
:1000D000003F000000000030003000000000000081
:1000E0000000300630060000000080008000800024
:1000F0008000800080000000000000000000000080
:1001000000001027E80364000A000100A81F200176
:10011000DA028D14AFA1C80E0C0DFF121112FF0EE2
:100120000A0DFF0E0A12FF0E0C12FF0E0B12FF003B
:1001300011241FBECFE5D2E0DEBFCDBF20E0A0E698
:10014000B0E001C01D92A436B207E1F73CD163C311
:1001500057CF282FB89898E080E0880FBA98B099C8
:100160008160BA9A9150C9F72111B89ABA98BA9A8F
:100170000895B89ABA98B898089598E087FF02C091
:10018000B89801C0B89ABA98BA9A880F9150B1F746
:10019000B898BA98BA9A08951F93CF93DF93E82F2F
:1001A000EE0FEE0FEE0F880F880FCE2FC80F80E0F6
:1001B000E4DF80E0E2DFDCE0DC0F11E01C0FEC2F7D
:1001C000F0E0E25EFF4F8491D8DFC12FD113F5CF6D
:1001D00080E0D3DF80E0DF91CF911F91CECFB89A3E
:1001E000BA9ACBCFCF93DF93C82F80E8F8DF8C2F5C
:1001F000C4DFB898BA9881E8F2DF81E0AADFC82F9F
:1002000080E0A7DFD0E0DC2FCC27C82BB2DFCE0107
:10021000DF91CF910895CF93C82F88E7E0DF80E486
:10022000ACDF80E0CA3018F08F5FCA50FBCFB4DF7C
:100230008C2FB2DFCF919DCF0F931F93CF93DF937E
:100240008C0188E7CCDF80E498DFC0E0D0E0FE01DD
:10025000EA5FFE4F2591349180E00217130720F0EA
:100260008F5F021B130BF9CF97DF2296C630D105A3
:1002700071F7DF91CF911F910F917BCFEF92FF929A
:100280000F931F93CF93DF937C0188E7A8DF80E46F
:1002900074DF02E011E0C0E0D0E0F8012591349174
:1002A00080E0E216F30628F08F5FE21AF30AD1E04D
:1002B000F8CFD11103C0C43009F082E16DDFCF5F08
:1002C0000E5F1F4FC53049F7DF91CF911F910F91FE
:1002D000FF90EF904ECFCF93DF93EC0188E77FDF65
:1002E00080E44BDFFE0184918F3F19F055DF2196AA
:1002F000F9CFDF91CF913DCFCF93C82F88E76FDF44
:1003000080E43BDF8C2F48DFCF9133CFCF93DF9357
:10031000C82FD62F88E763DF80E02FDF82E22DDF52
:100320008D2F2BDF81E08D0F28DF8C2F8F7025DF45
:100330008C2F82958F70806120DF8D2F806B1DDF69
:10034000DF91CF9116CFCF9360E080E0DFDF88E7C9
:1003500046DF80E412DFC0E080E00FDFC150E1F74C
:1003600008DF62E080E0D2DF88E739DF80E405DF84
:1003700080E003DFC150E1F7CF91FBCE1F920F92D7
:100380000FB60F9211248F939F93AF93BF938091D9
:10039000600090916100A0916200B09163000196AD
:1003A000A11DB11D8093600090936100A093620035
:1003B000B0936300BF91AF919F918F910F900FBE4B
:1003C0000F901F901895CF93DF93CDB7DEB7A4970A
:1003D0000FB6F894DEBF0FBECDBFC39A8CE789BDC0
:1003E00082E08ABD83BF80E189BF80E8F8DE80E0DB
:1003F000C4DE87E0C2DE8FEFC0DEBBDE80E8EFDE6A
:1004000085E0BBDE84E1B9DE80E0B7DEB2DE88E7FE
:10041000E6DE80E0B2DE2CE031E03C832B8307E1B6
:1004200011E0EB81FC818491A8DE2B813C812F5F60
:100430003F4F3C832B830217130799F79ADE83DF24
:10044000F894C0906000D0906100E0906200F0905D
:100450006300789431E03A831982198A1A8A1B8AD8
:100460001C8A412C512C32011D861E861F86188A3B
:100470001C861B864FEF5FEF5A87498718861F82BD
:100480008FEF9FEF9E838D83212C312CAFEFBFEF39
:10049000BC83AB8338EE832E33E0932EA12CB12C9A
:1004A00082E0A0DE969587958C010C7F84E09ADE31
:1004B0009CA38BA397FF02C01CA21BA2F8942091BF
:1004C00060003091610040916200509163002F8F75
:1004D00038A349A35AA378942C193D094E095F0902
:1004E0002D8B3E8B4F8B588F8D859E85AF85B88920
:1004F000820F931FA41FB51F8D879E87AF87B88B70
:10050000ABA1BCA1AD0160E070E0C801A0E0B0E02B
:10051000498F5A8F6B8F7C8F9A01AB01BC01CD0143
:100520002BD1A501940155D169017A013E8F2D8F00
:10053000298D3A8D4B8D5C8D6D897E898F89988D43
:100540001BD120E13EE040E050E043D1420E531E7B
:10055000641E751EC701B601882799272D893E891B
:100560004F89588D09D120E13EE040E050E031D183
:1005700089899A89AB89BC89820F931FA41FB51FF3
:10058000898B9A8BAB8BBC8BAB81BC810A171B0709
:1005900010F41C830B832016310608F41801ED813A
:1005A000FE812BA13CA12E173F0710F43E832D8323
:1005B0004F8158858BA19CA14817590710F4988743
:1005C0008F83A985BA85ED8DFE8DEA17FB0710F4A0
:1005D000DA86C9862B853C854D8D5E8D24173507BF
:1005E00010F4DC86CB86B3990DC05A8151110CC032
:1005F00089818F5F8983853008F01982A4DE91E0BC
:100600009A8304C01A8202C0A1E0AA83B981B230E1
:1006100009F46FC018F5BB2309F44BC0B13009F0E1
:10062000A0C060E080E072DE8B819C8127DE8BE1E0
:1006300091E051DEC10122DE8BE291E04CDE62E00E
:1006400080E064DE8D819E8119DE8BE191E043DEE6
:100650008F81988513DE83E291E059C0E981E33010
:1006600009F457C0E43009F07CC06D857E858F8524
:100670009889A5019401ADD03E8B2D8B61E080E27D
:1006800045DE8D899E8960E17EE08FD09E8B8D8BCB
:10069000862FC1DD80E130DE8D899E896CE370E0BC
:1006A00084D08D8B862FB7DD80E126DE8D89B3DD8A
:1006B00058C060E080E02ADEC801E0DD8BE291E016
:1006C0000ADEC601DBDD87E291E005DE62E080E064
:1006D0001DDE8BA19CA1D2DD83E291E0FCDDC30194
:1006E000B201A501940175D0C901C8DD8FE191E087
:1006F0000EC061E080E00ADE89859A85BFDD8BE16E
:1007000091E0E9DD8B859C85B9DD87E291E0E3DD51
:1007100028C060E080E1FADDC301B201A5019401C7
:1007200058D06B017C01C901A9DD8FE0E5DDC60170
:1007300083DD8FE191E0CFDD62E080E1E7DD698973
:100740007A898B899C89A501940143D06B017C0136
:10075000C90194DD8FE0D0DDC6016EDD87E191E057
:10076000D6CF83ED90E30197F1F700C00000CF8C66
:10077000D8A0E9A0FAA094CEEE27FF27AA27BB278E
:1007800008C0A20FB31FE41FF51F220F331F441F21
:10079000551F969587957795679598F37040A9F7BB
:1007A000009799F7BD01CF010895AA1BBB1B51E12A
:1007B00007C0AA1FBB1FA617B70710F0A61BB70BD1
:1007C000881F991F5A95A9F780959095BC01CD0176
:1007D0000895A1E21A2EAA1BBB1BFD010DC0AA1F82
:1007E000BB1FEE1FFF1FA217B307E407F50720F09A
:1007F000A21BB30BE40BF50B661F771F881F991F15
:100800001A9469F760957095809590959B01AC015D
:0A081000BD01CF010895F894FFCF59
:00000001FF
